:020000040800F2
:10500000081C0020D5500008F58F00082B860008EA
:105010000000000000000000000000000000000090
:105020000000000000000000000000004D9C00088F
:1050300000000000000000002D9A0008899D000873
:10504000E7500008E7500008E7500008E750000864
:10505000E7500008115C0008E7500008E75000081E
:1050600000000000E75000081D5B0008E750000842
:10507000E7500008058B000800000000E75000081A
:1050800000000000E75000080000000000000000E1
:10509000E750000800000000E7500008E750000853
:1050A000E7500008E7500008E75000081DA8000876
:1050B000E7500008E7500008000000000000000072
:1050C0000348854600F074FC00480047FDB800081E
:1050D000081C00200448804704480047FEE7FEE71C
:1050E000FEE7FEE7FEE7FEE7499E0008C150000824
:1050F00030B50B46014600202022012409E00D4670
:10510000D5409D4205D31D469540491B25469540F7
:1051100040191546521E002DF1DC30BD70B500243B
:105120002546002801DA01244042002901DA012540
:105130004942FFF7DDFFAC4200D04042002C00D0D6
:10514000494270BDF0B51FB40646002082B0054646
:105150004024019100901BE0019922460F46304601
:1051600000F062FB049A059B801A994110D3104607
:105170001946224600F048FB361A8F410197224615
:1051800001200021009F00F03FFB38184D410090A6
:105190002046641E0028DFDC019B00982946324629
:1051A00007B0F0BD03460B439B0703D009E008C9D5
:1051B000121F08C0042AFAD203E00B780370401CC7
:1051C000491C521EF9D27047D2B201E00270401C55
:1051D000491EFBD270470022F6E710B513460A4677
:1051E00004461946FFF7F0FF204610BD30B50446CF
:1051F0000020034600E05B1C934203D2E05CCD5CE0
:10520000401BF8D030BDF8B502464A40D40F4200EA
:105210004B0052085B089A4202D2024608461146E9
:105220004A0023D0C30D4A00DDB2120EAD1A202D64
:1052300035DA49020126490AF6058A19002C00D000
:10524000524220214F1B1146B9402A411018C20D6D
:105250009A4221D0002C17D0012D08DCDA05801AE3
:10526000D20F8019D207DBB200F00AFBF8BDDA05D5
:10527000801A012340001B06C01880185A4280186B
:10528000CA0F1043490007E04908C2071143DA0575
:10529000801A80194008801800F0EAFAF8BD610011
:1052A0000122511A001BF7E70122D2075140AAE759
:1052B0000122D2075040A6E770B502464A40D50FFA
:1052C00040004A00ED0740085208002814D0002A88
:1052D00012D0C40DD30D41020120C0055202490A6B
:1052E000520AE41A091812187D34914201D3641C41
:1052F00000E04900002C01DA002070BD002391423B
:1053000001D3891A0343400849000028F7D1002936
:105310000AD0914202D10121C90705E0914201D290
:10532000012101E00121C943E005C018401900F046
:105330009FFA70BDF0B507460846584087B0C00FC9
:10534000049048000E46590040084908BC1A88419C
:1053500005D2384631461E4617460B4602465800CF
:10536000400810434CD0300D039040055900400DCB
:10537000490D0590401A0290402872DA1803012165
:10538000000B09050843019004980092002805D0FD
:1053900001995242002088410092019002984021D8
:1053A0000A1A0199009800F02FFA05460C466B4640
:1053B00007CB00F04AFAC0197141039A0E0D002381
:1053C000D71756401A467A40164344D0049A002A0A
:1053D0002DD0029A012A039A15DC1205C01A9141B8
:1053E00001263605001C7141D20F059ED20700939D
:1053F000019202962A46234600F088FA07B0F0BDD3
:1054000038463146FAE71605224A0F46B218C01A46
:10541000B74101210905001C4F4100187F41114689
:1054200018187941E20F10436D19644113E0E20747
:105430006D0815436408C2071443039A0126120538
:10544000C01A91413605001C7141CE074008304317
:105450004908C01851412A46234600F04AFACDE7D0
:10546000FFE7049801224000C117121A00238B4164
:1054700004983146C417381AA141EEE730B401242C
:10548000E407634030BC55E730B40124E4076140D1
:1054900030BC4FE70000E0FFF0B51FB488B00B99B7
:1054A0000998002448400999C00F4900490809910A
:1054B000C0070B990090490049080B910999089879
:1054C000A64608431CD00B990A98084318D009989F
:1054D00001244000420D4800410D099824050003B5
:1054E000000B204309900B980003000B20430B9006
:1054F00050181C494018002201901446104605E03F
:10550000002001460DB0F0BD032801DA034600E09B
:1055100003239C46C11A0AAE0AE05F0008ADED5BAA
:105520004F00F75B7D430027AA187C41491C5B1E96
:105530006145F2DD410004AB5A522104120C0A43CA
:10554000240C401C0828DFDB01980290009970466B
:1055500001910090059B049A0799069800F0D6F9EE
:10556000D0E700000DFCFFFFF0B50C465C4085B0B5
:10557000E40FE40703944C000026640859009446A5
:10558000490802460296224321D062460A431ED0B1
:105590006200570D4A000E032303550D01240246F5
:1055A0002C492405781B1B0B360B4018234326433C
:1055B000614600901C46501AB44103D30098401C29
:1055C000009002E0921800985B41002803DA002066
:1055D000014605B0F0BD00200121090507468646B9
:1055E00011E064461D46141BB54106D36546521BA7
:1055F000B341744607430C43A646CD07400849080B
:10560000284392185B4105460D43EAD110461843E2
:1056100013D06046194650407140084306D060469A
:10562000101AB34106D20122002306E00022012312
:10563000DB0702E00122D2435310009874460105B3
:10564000381C6141029C039D0019694100F051F929
:10565000BFE70000FD03000010B5002296231146AD
:1056600000F00EF910BD00000EB5C217C10F50407A
:10567000CA0740180021054B0293019200910A4687
:105680000B4600F043F903B000BD000033040000F6
:105690000EB505490291002100910A460B46019181
:1056A00000F034F903B000BD3304000041004002B3
:1056B0000122400AD205090E80187F2901DA002054
:1056C0007047962903DC9622511AC84070479639D4
:1056D0008840704770B5CD0F4A0009030123090BBC
:1056E0001B0519430B4BED070024520D9A4201DABA
:1056F000002070BD074B34339A4203DC9A1A00F045
:1057000093F802E00449511888402C43F1D04042FC
:1057100070BD0000FF030000CDFBFFFF4A0009033E
:105720000123090B1B051943094B10B5520D9A4271
:1057300001DA002010BD064B34339A4203DC9A1A7A
:1057400000F072F810BD03495118884010BD0000E8
:10575000FF030000CDFBFFFFC20FD207400040084F
:105760000BD0C10D0723DB01C91840020905400A0F
:105770001143C2084007114370470020014670479B
:1057800010B5002904DB0124E40740428C41214686
:10579000002B04DB1C460123DB075242A341994244
:1057A00000D1904210BD0000CB0FDB07490010B5BF
:1057B000490802460A4307D00A0D07240903E401F9
:1057C000090B121B002A01DC002010BDC900440F88
:1057D0000C43C100E018D205801800F049F810BD54
:1057E0000122D207002800DB101A002900DB511A21
:1057F000814270470122D207002800DB101A0029DD
:1058000000DB511A8842704710B5202A04DB01469C
:10581000203A9140002010BD914020239C1A03465D
:10582000E3401943904010BD10B5202A04DB084620
:10583000203AD040002110BD0B46D340D040202458
:10584000A21A91400843194610BD10B5202A06DB64
:10585000CB170846203A1041C1170B4306E00B4610
:105860001341D0402024A21A91400843194610BD8C
:10587000002904DA401C490001D14008400070476B
:1058800070B40024050C05D11024000402D10029B5
:1058900021D01124050E01D100020834050F01D1D9
:1058A0000001241D850F01D18000A41C002801DB0C
:1058B0004000641C002908D020252E1B0D46F54011
:1058C000A14000D001212943084301061B1B000A07
:1058D000DB1D02D5002070BC7047DB05181880184E
:1058E0000029F8DA401C4900F5D170BC400840009E
:1058F000704710B5002B08DA0024401C6141921853
:105900005B411A4301D14008400010BDF0B51FB4FF
:1059100082B005460C0003D0084605F08FF802E07F
:1059200005F08CF820300246009021462846FFF70B
:105930006BFF049B059A04460F4618431143084326
:1059400014D0184610431BD0009840210A1A18465C
:105950000599FFF769FF05460E46009A05990498D8
:10596000FFF752FF084305D0012004E020463946E6
:1059700007B0F0BD0020C11705430E432C43374349
:1059800000990E986305401A7905E40A00220C4339
:10599000FD0A0A3002D500200146E9E70105101989
:1059A00069410C9C0D9D00196941FFF7A2FFDFE7DB
:1059B000064C0125064E05E0E36807CC2B430C3C62
:1059C00098471034B442F7D3FFF77EFBCCBC0008F5
:1059D000ECBC000870B58C180578401C6B075B0F99
:1059E00001D10378401C2A1106D10278401C03E043
:1059F00006780E70401C491C5B1EF9D12B0705D49C
:105A00000023521E0DD40B70491CFAE70378401C8A
:105A1000CB1A921C03E01D780D70491C5B1C521EB2
:105A2000F9D5A142D8D3002070BD000038B5044696
:105A3000074908480068FFF75BFB6043009002E0FD
:105A40000098401E009000980028F9D138BD000051
:105A500040420F008001002070B5044600252068F8
:105A600080688007800F012807D120680068C00780
:105A7000C00F002801D0012000E00020002839D10B
:105A8000206880681C490840002801D1012000E0FE
:105A90000020002809D1606D102108436065A06DC9
:105AA00001210843A065012070BD206880680121A4
:105AB0000843216888600120FFF7B8FF01F012FA5F
:105AC00005460EE001F00EFA401B0A2809D9606D68
:105AD000102108436065A06D01210843A0650120E5
:105AE000E2E720680068C007C00F01214840484035
:105AF0000028E7D00020D7E71700008010B5024645
:105B00000B460020002103E0545C2418A0B2491C7D
:105B10009942F9D3C443A0B210BD000010B50348A8
:105B200000F0DEFE024800F0DBFE10BDA4170020EE
:105B30005C17002030B51C25446C2C400125A54085
:105B4000046C6560046863608468102C04D1046888
:105B5000A2600468E16003E00468A1600468E26098
:105B600030BD0000012017494872022016494872D2
:105B700003201649487204201549487211481549F6
:105B80000A78427149788171104812490A78427145
:105B9000497881710C480F490A78427049788170C0
:105BA0000B480C490A784270497881700A480949C3
:105BB0000A7842704978817006490A7842714978BA
:105BC00081717047B411002012120020D6110020FC
:105BD000C81100203C0100202812002010B504F05C
:105BE00009F8202004F0BEF8012005F043FB002056
:105BF00004F0B8F8044805F0ABF9044805F0EAFCF5
:105C0000002005F027FD10BD61000020838000000A
:105C100010B501210520000701F054F9002802D039
:105C200000200B49086002210A4801F04BF90028C6
:105C300007D107490860084800880A2148430749F6
:105C40000880012001F038F8022001F035F810BD7D
:105C50007801002000040050580100206801002055
:105C60007047000000210A4A51610A49496801222F
:105C700052021143074A51601146496808221143F4
:105C8000044A51600021C209D2011160704700002E
:105C9000EC170020002002407FB504460D4600208E
:105CA000039000F0C1FF002000900194E8090290E9
:105CB00003A9684600F03AFF002804D000F07CFFFA
:105CC000002004B070BD00F077FF0120F9E710B5A7
:105CD0000346002002E01C5C0C54401C9042FAD3A6
:105CE00010BD0000002039498969FF2201321140AE
:105CF000914208D13649496902221143344A51611F
:105D0000FF210131084331498969012252021140C2
:105D1000914208D12E494969012211432C4A51610F
:105D2000012149020843294989690122920211404F
:105D3000914208D12649496908221143244A5161F8
:105D4000012189020843214989690122D2021140B7
:105D5000914208D11E494969042211431C4A5161EC
:105D60000121C902084319498969012252031140DE
:105D7000914208D11649496910221143144A5161D0
:105D80000121490308431149896901225204114044
:105D9000914207D10E494969202211430C4A5161B1
:105DA00020210843094989690122120411409142C6
:105DB00008D10749496940221143054A516101212F
:105DC000090408430149886170470000002002402F
:105DD000EC17002070B5044601F084F805460BE08E
:105DE000601C002808D0002C04D001F07BF8401B78
:105DF000A04201D9032070BD1F488069C007C00FB1
:105E00000028EDD11C48806902210840022801D1F8
:105E10001949886118488069FF210131084088428A
:105E200023D0154880694900084088421DD0124897
:105E3000806949000840884217D00F4880694900AE
:105E40000840884211D00C48806989000840884287
:105E50000BD00948806909010840884205D00648EE
:105E6000806949100840884203D1FFF73BFF0120B9
:105E7000C1E70020BFE7000000200240F0B585B078
:105E800006460F4614460025029601970020009012
:105E900000F0CAFE13E00198006803900220039A04
:105EA000029900F099FE00900098002800D008E0C8
:105EB0000298001D02900198001D01902D1DA54221
:105EC000E9D300BF00F078FEA54202D2002005B061
:105ED000F0BD0120FBE700000246002108E0480079
:105EE000064B185A904201D108467047481CC1B26F
:105EF000034800788142F2DB00BFF6E7221400205D
:105F000028010020FEB50C4801F0D0F980B20290C3
:105F10000298FFF7BDFB0446084A094BFFF7BCFA9D
:105F20000022084B01910090FFF71EFB0646FFF789
:105F3000F5FB80B2FEBD000054160020F853E3A527
:105F40009B843E4000408F4010B54B4800780028AD
:105F500003D000204849087002E00120464908703B
:105F6000464845490A7842704978817044490A7820
:105F7000427149788171052040494872962005F0A8
:105F800017FB4B20C00005F02FFB00223B490C20E3
:105F900005F02CFC00210C2005F03CFC022005F053
:105FA00061FB00BF00210F2005F05AFA3549086057
:105FB000354908400028F5D032480068401C0028C8
:105FC00001D103F055F82F480068012189030840EA
:105FD00000283FD08122D20100210F2005F0BFFB15
:105FE0000021102005F03CFA4406640E21460022F0
:105FF000264805F085FA2548407A05283AD102223C
:106000001F492248401DFFF7F1F8002832D11F48F0
:10601000807A1F49087004221C49491C1D48FFF75B
:10602000C1F81C48006800F043F81B490880184874
:106030000078420015490B311848FFF7B3F81648AD
:1060400000881749098848431649088002201649E4
:1060500008700FE0104908880988491E0E4B198006
:1060600012490988FFF75AF80D480088414388B261
:106070000C49088010BD00003401002028120020C7
:106080003C0100207000002000D02724781200205E
:10609000280100202C010020FC00002022140020F8
:1060A0004E0100204A010020600000205001002025
:1060B00070B50646174801F0F9F8C5B22846E91749
:1060C000C90E091849114901691ACCB209E03046D4
:1060D000E040C007C00F002801D1204670BD601C01
:1060E000C4B20D4800888442F1DB012409E0304647
:1060F000E040C007C00F002801D12046EEE7601C39
:10610000C4B2054800888442F1DB03480078401E91
:10611000C0B2E3E7541600205001002010B50B4830
:1061200000F074FB0A21094800F0FAFA074800F071
:10613000A1F9012149020840884204D1034800F036
:106140009CF980B210BD00BFFCE70000F8150020EC
:10615000F0B587B000220121424800F0BCFEFFF7F5
:10616000DDFF0546FFF778FA04463F49FFF7A4F83C
:106170003E490860012211463A4800F0ACFE3B4817
:106180000068FFF7E9FA04460022394BFFF7F8FAF6
:106190005ED838480078002821D0002035490870A2
:1061A000FFF7BCFF0546FFF757FA04462E49FFF7F5
:1061B00083F82E49086008460068FFF7CDFA0446C8
:1061C00000222B4BFFF75AF900222B4B059104902C
:1061D000FFF762F90646FFF7E7FA28490860234807
:1061E0000068FFF7B9FA06460022214BFFF746F98F
:1061F0000446234A234BFFF74FF9039102901F48AF
:106200000068FFF7A9FA04461D4A52421E4BFFF7E9
:1062100043F901910090039B029AFFF78BF80591D7
:106220000490FFF7C1FA154908601849134800683F
:10623000FFF7E0FA02D215481049086000210F4824
:106240000068FFF7CDFA06D200200C49086002E092
:1062500000200A49086009480068FFF727FAC0B221
:1062600007B0F0BD0004005000401B44280000208F
:1062700000000C403000002000E064402C000020B2
:106280003333333333B33040CCCCEC3F0000C8421F
:10629000F8B5044600250026002700BF5020005D09
:1062A000012801D10220F8BD01215020015500BF75
:1062B000206880688007800F012806D12068006868
:1062C0000840002801D0012000E00020002841D132
:1062D000606DFF2101318843022108436065206819
:1062E000C0688707BF0F2068C068800880002168E9
:1062F000C860206880680121C90708432168886058
:1063000000F0F0FD064611E000F0ECFD801B0A28CD
:106310000CD9606D0221884310210843606500BFDD
:1063200000215020015500BF0120BCE72068806893
:10633000C00FC0070121C9078842E5D02068C068A6
:1063400038432168C860606D0221884301210843F9
:10635000606504E0606D202108436065012500BF91
:1063600000215020015500BF28469CE770B5044627
:106370000D4600BF5020005D012801D1022070BDF4
:1063800001215020015500BF206880680421084089
:10639000800800280AD0606D20210843606500BF96
:1063A00000215020015500BF0120E8E72D49686811
:1063B000884229D02068806A29684903490B08432C
:1063C0002168886228684003400B27490840012162
:1063D0008904884208D12548806849010843234937
:1063E00088600A20FFF722FB28684003400B204901
:1063F00008400121490488422CD11C488068490189
:1064000008431A49886025E02068806A29684903A2
:10641000490B88432168886228684003400B124971
:10642000084001218904884205D11048806849014B
:1064300088430E49886028684003400B0C49084097
:1064400001214904884205D10848806849018843F0
:106450000649886000BF00215020015500BF002080
:106460008DE70000011000000000044800270140F3
:10647000000002440146486D704701460868006C00
:106480007047000010B50446002C01D1012010BD5A
:10649000606D002806D1A0650021502001552046DE
:1064A00000F00EF9606D10210840102806D0206819
:1064B000806804210840800800280AD0606D1021FF
:1064C0000843606500BF00215020015500BF012036
:1064D000DDE7606DFF2101318843022108436065DB
:1064E000206880688007800F012807D12068006835
:1064F000C007C00F002801D0012000E000200028C4
:106500003AD100BF032189076068884207D0494219
:106510006068884203D04900606888420CD12068D6
:10652000006980008008216808612068006961684E
:1065300008432168086112E0206800698000800833
:10654000216808615C4880680F21890488435A49A2
:10655000886008468068616808435749886000BFC2
:106560002068C068182188432168C8602068C06816
:10657000A16808432168C8604F4880680121490626
:1065800088434D49886008468068A18E49060843C3
:10659000494988602068806801210907084000286F
:1065A00004D1206880680843216888602068C0683A
:1065B000424908402168C8602169E068022901D188
:1065C000042100E0002108432021095D490308431C
:1065D0002C21095D49000843216B0843A169890307
:1065E0000843E169C90308432168C9680843216871
:1065F000C860FF21C231606A884207D0A16A606A20
:1066000008432168C96808432168C8602120005DEB
:10661000012813D12020005D002807D12068C06820
:106620000121090408432168C86007E0606D20214A
:1066300008436065A06D01210843A065E06B012857
:1066400017D120680069FF2189008843216808610B
:10665000216C606C0843A16C0843216809690843F8
:1066600021680861206800690121084321680861E8
:106670000BE020680069C007C00F002805D0206823
:106680000069400840002168086120684069C0082E
:10669000C0002168486120684069A16B08432168F7
:1066A00048610020A065606D0221884301210843F4
:1066B00060650020EBE60000002701401902FEFFA4
:1066C00010B586B00446142101A8FEF784FD1249D6
:1066D000206888421ED11148406B491508430F4974
:1066E000486300BF0846C06A012108430B49C862DD
:1066F0000846C06AC007C00F009000BF00BF02205C
:106700000190032002900020039001A905200007BA
:1067100000F0E2FA06B010BD002401400010024073
:10672000F8B504460D46002600276069082801D107
:10673000082711E02068C068C007C00F00280AD0F1
:10674000606D20210843606500BF00215020015585
:1067500000BF0120F8BD0C2700F0C4FB064614E082
:10676000681C002811D0002D04D000F0BBFB801B5A
:10677000A8420AD9606D04210843606500BF00216A
:106780005020015500BF0320E4E72068006838402E
:106790000028E5D0606D012149020843606520684A
:1067A000C068032189020840002826D12020005D0E
:1067B000002822D1206800680821084008281CD140
:1067C0002068806804210840800800280DD12068D6
:1067D00040680C21884321684860606DFF210131C9
:1067E000884301210843606507E0606D202108436C
:1067F0006065A06D01210843A065A069002802D151
:106800000C20216808600020A4E7000070B5044651
:1068100000252068806804210840800800282BD1CA
:1068200000BF5020005D012801D1022070BD012170
:106830005020015500BFE069012803D02046FFF732
:106840000BF90546002D18D1606D0D490840FF2158
:106850000131084360650020A06500BF0021502081
:10686000015500BF1C202168086020688068042151
:1068700008432168886000E002252846D6E700002A
:10688000FEF1FFFF70B5044600252520005D0228BB
:1068900003D00420E063012520E0206800680E2179
:1068A000884321680860206800684008400021682B
:1068B00008601C21606C084001218140206C41600F
:1068C00001212520015500BF00212420015500BFD2
:1068D000A06B002802D02046A16B8847284670BDD7
:1068E00070B50446206C0568206806681C20616C41
:1068F000014004208840284000281DD0042030405A
:10690000002819D02068006820210840002805D1FF
:106910002068006804218843216808601C21606C9D
:10692000084004218140206C4160206B00285AD02F
:106930002046216B884756E01C20616C01400220F4
:1069400088402840002825D002203040002821D04F
:106950002068006820210840002808D120680068CD
:106960000A218843216808600121252001551C2146
:10697000606C084002218140206C416000BF002112
:106980002420015500BFE06A00282CD02046E16A8F
:10699000884728E01C20616C01400820884028407E
:1069A000002820D00820304000281CD02068006833
:1069B0000E218843216808601C21606C0840012179
:1069C0008140206C41600120E063012125200155B8
:1069D00000BF00212420015500BF606B002802D0B9
:1069E0002046616B884770BD70B50446002C01D10C
:1069F000012070BD244A2168881A1421FEF778FB13
:106A00008000606420480838206402212520015558
:106A1000206805681D480540E168A06808432169B1
:106A2000084361690843A1690843E1690843216A91
:106A3000084305432068056001218903A068884256
:106A400017D011487830806A1C22616C11400F22E7
:106A50008A4090430C49783188621C22616C114055
:106A60006068884008497831896A08430649783166
:106A700088620020E06301212520015500212420A7
:106A800001550020B5E70000080002400F80FFFF1D
:106A9000F8B504460D4616461F460020009000BF7C
:106AA0002420005D012801D10220F8BD012124200D
:106AB000015500BF2520005D01282DD10221252090
:106AC00001550020E063206800684008400021680C
:106AD00008603B46324629462046FFF72BF8206BDC
:106AE000002806D0206800680E210843216808604D
:106AF0000BE0206800680421884321680860206852
:106B000000680A21084321680860206800680121A4
:106B100008432168086006E000BF002124200155D9
:106B200000BF022000900098BFE70000F8B50446BF
:106B30000E460127002500BF1C48007C012801D11A
:106B40000220F8BD01201949087400BF1848FFF75A
:106B500041F90746002F22D1401E3060656817E0DA
:106B60002846FFF77FF81248FFF734F90746114827
:106B70004068082188430F49486008464068491525
:106B800088430C494860002F01D0356006E080350D
:106B9000A068C00161684018A842E1D800BF00BFEA
:106BA00000200249087400BF3846CAE7EC170020ED
:106BB00050C30000002002400648406802210843FC
:106BC000044948600846406801210843014948607B
:106BD0000020704700200240F8B507460C461546D5
:106BE000012600BF0E48007C012801D10220F8BD1B
:106BF00001200B49087400BF0A48FFF7EBF806466E
:106C0000002E06D10649486125600648FFF7E2F8E4
:106C1000064600BF00200249087400BF3046E6E780
:106C2000EC17002050C300001D484068C007C00F8B
:106C3000002816D000BFEFF31080014600BF72B6E7
:106C40001848174AD0601848D06000BF81F31088F8
:106C500000BF10464068C007C00F002801D00120C7
:106C600070470F48406802221040022815D100BF2B
:106C7000EFF31080014672B60C48094A10610C48C7
:106C80001061084680F3108800BF10464068022259
:106C90001040022801D10120E2E70020E0E70000D7
:106CA00000200240EFCDAB8905040302BFAE9D8CEE
:106CB000161514137047000010B5044605484069C6
:106CC0002040002804D0034844612046FFF7F2FF2B
:106CD00010BD00000004014070B5034600220024EE
:106CE0000020DAE0012696400D6835402C46002C45
:106CF00077D04D68022D02D04D68122D15D1D508E0
:106D0000AE001D462035A8595507EE0E0F25B5409B
:106D10000646AE4330465607F60E0D69B540284389
:106D2000D508AD001E46203670514D68012D08D0A3
:106D30004D68022D05D04D68112D02D04D68122DE1
:106D400018D1986856000325B5400646AE43304634
:106D50005600CD68B5402843986058680125954095
:106D60000646AE43304610264D6835402D09954005
:106D700028435860186856000325B5400646AE43C0
:106D800030460D79AD07AD0F5600B5402843186069
:106D9000D86856000325B5400646AE433046560037
:106DA0008D68B5402843D860012636074D683540C8
:106DB000B54271D13C4D6D6B012635433A4E75633A
:106DC0003A4D9608B600A85995072E0F0F25B540E5
:106DD0000646AE43304605252D07AB4202D10025BD
:106DE00015E059E0324DAB4201D101250FE0314DA4
:106DF000AB4201D102250AE02F4DAB4201D1032560
:106E000005E02E4DAB4201D1052500E00625960791
:106E1000360FB5402843254D9608B600A851284D99
:106E200028680546A5432846012636044D683540A6
:106E3000B54202D1054625432846214D28606868A1
:106E40000546A5432846012676044D683540B542DF
:106E500002D1054625432846194D6860A8680546B5
:106E6000A5432846012636054D683540B54202D176
:106E7000054625432846124DA860E8680546A54307
:106E80002846012676054D683540B54202D10546B3
:106E9000254328460A4DE860521C0D68D540002D58
:106EA00000D01FE770BD0000001002400800014044
:106EB0000004005000080050000C0050001C00505E
:106EC00000040140024613690B40002B01D0012051
:106ED00000E000207047002A01D0816100E081625B
:106EE0007047000001480068704700007C010020E6
:106EF00002480068401C0149086070477C0100207E
:106F000010B500240848006840210843064908607D
:106F1000002000F00BF8002801D0012401E000F06F
:106F2000FBF9204610BD00000020024070B5044669
:106F300000257D21C90009480068FEF7D9F80646FA
:106F400001F0AAF8002801D0012504E00022214622
:106F5000501E00F009FA284670BD00008001002094
:106F60007047704770B505462A480078401C29498B
:106F7000087001202849087028480088401C2749CB
:106F800008802748008802F0A5FE2649C888FEF739
:106F900063FB06462449FEF78FF90446234801683F
:106FA0002046FEF730F92149086002212048FFF70A
:106FB00089FF002819D11B49C888FEF74DFB0646FA
:106FC0001949FEF779F904461A4801682046FEF788
:106FD0001AF918490860184916480068FEF70AFCB3
:106FE00006D816481649C86002E00020114908601A
:106FF0000C49488FFEF730FB04460C4801682046D8
:10700000FEF7EEFB05D20F480078002801D004F00F
:107010000BFD70BD740100204901002062010020B9
:107020004A010020B40D002000007A4478010020BD
:10703000000400506C0100200000A0400400FA058C
:1070400000ED00E05E010020704710B50446002C02
:1070500001D1012010BD02212E200155204601F052
:1070600059FD204600F0F4F800212E20015500BF04
:107070002D20015500BF0020ECE77047704710B588
:10708000044620680068C007C00F012148404840FE
:1070900000280CD0206880680840484048400028FC
:1070A00005D00120216848602046FFF75BFF20687B
:1070B000006802210840400800280BD02068806842
:1070C00008404008002805D002202168486020467A
:1070D000FFF746FF20680068042108408008002868
:1070E0000BD02068806808408008002805D0042064
:1070F00021684860204600F00DF9206800680821EA
:107100000840C00800280BD0206880680840C008EC
:10711000002805D00820216848602046FFF794FF2A
:107120002068006810210840000900280BD0206862
:10713000806808400009002805D0102021684860B8
:107140002046FFF70EFF2068006820210840400914
:1071500000280BD02068806808404009002805D02E
:107160002020216848602046FFF788FF20680068DB
:1071700040210840800900280BD020688068084022
:107180008009002805D04020216848602046FFF78C
:1071900074FF10BD70B50446002C01D1012070BDF4
:1071A0006068012800D100BF26496069884200D08C
:1071B00000BF2E20005D002805D100212D200155A3
:1071C000204600F059F802212E2001552068C5689C
:1071D0006068012803D08905A06A884203D11E2176
:1071E00028468843054617496069884201D01648F9
:1071F000054016480540A16860680843216A0843B5
:10720000616A0843A16A084305436068012804D005
:107210000121C905A06A884203D1E16820690843B9
:10722000054308496069884205D06169A06908433F
:10723000E169084305432068C56001212E200155FE
:107240000020ACE7FFFF00003F1FFFFFF8F119FF30
:1072500010B5044606492068884208D10548806B6D
:1072600040004008034988630D2000F065F810BD18
:10727000007C00400010024010B504460949206817
:1072800088420DD10848806B490508430649886348
:10729000002201210D2000F067F80D2000F058F8C1
:1072A00010BD0000007C004000100240014608684C
:1072B000C069704710B5034602242E20C4541448F8
:1072C000006824072043124C20601868C06801241D
:1072D000E40420431C68E0601868806801242043AF
:1072E0001C68A06018680069012420431C682061A4
:1072F0001868816118684261186800690424204395
:107300001C68206101242E20C454002010BD000000
:1073100000040140704700000648406B012108430B
:10732000044948630846806B09040843014988639F
:10733000704700000010024000BFC206D20E0121BB
:107340009140024A116000BF7047000080E100E0F8
:1073500000BFC206D20E01219140024A116000BF57
:107360007047000000E100E070B504460D46164687
:107370002946204601F040FE70BD000002494968E0
:107380008143014A51607047007000400348006823
:10739000FF21013108430149086070470070004037
:1073A000024949680143014A51607047007000403A
:1073B000074800680221084305490860054800693C
:1073C000042108430349086100BF00BF30BF704774
:1073D0000070004000ED00E010B5024600200E4BAA
:1073E0001868800880000346134318460A4B18604B
:1073F0000A4B1B6904242343084C2361012901D152
:1074000030BF02E040BF20BF20BF044B1B690424F3
:10741000A343024C236110BD0070004000ED00E06A
:10742000F8B5044620212068084020287CD1206837
:107430000840202800D100BF00278148806B01212F
:1074400009070840002805D17D48806B08437C4926
:10745000886301277B480068FF210131084000282C
:1074600016D178480068084376490860FFF73AFD6E
:10747000064606E0FFF736FD801B642801D903208D
:10748000F8BD70480068FF21013108400028F1D0A4
:107490006B480568032109050D4060680840A84253
:1074A0000DD0091160680840884208D1644800681E
:1074B000012149040840884201D10120E0E76048E9
:1074C000403000690321090408400546002D3DD0E5
:1074D00060680840A84239D0202120680840202850
:1074E00034D15748403000690321090488430546D8
:1074F0005348403000690121C904084350494031D4
:107500000861084600690121C90488434C4940319B
:10751000086108460561801528408915884215D103
:10752000FFF7E0FC064608E039E0FFF7DBFC801BD4
:107530004549884201D90320A2E74148403000690B
:10754000012149020840400A0028EED000BF00BFD8
:10755000032109046068084088420AD1384800685D
:107560000901884303221205616811400843344928
:10757000086000BF3248403000690322120461688D
:10758000114008432E494031086100BF012F05D149
:107590002B48806B890588432949886300BF207880
:1075A000C007C00F002809D025484030C0688008B7
:1075B0008000A168084322494031C8600221206848
:1075C0000840022809D11E484030C0680C21884379
:1075D000E16808431A494031C86004212068084026
:1075E00004280AD116484030C06803218902884324
:1075F0002169084312494031C860082120680840C9
:1076000008280AD10E484030C06803210903884386
:10761000616908430A494031C860802120680840F8
:1076200080280AD106484030C06803218904884375
:10763000A169084302494031C860002020E70000EA
:10764000001002400070004088130000F8B50446A6
:107650000D46002C01D10120F8BD79480068C00713
:10766000C00FA8420ED27648006840084000284368
:107670007349086008460068C007C00FA84201D0DF
:107680000120E9E7022120680840022807D16D485F
:10769000C068F0218843A16808436A49C86020781F
:1076A000C007C00F00284CD06068022809D1654887
:1076B0000068012149040840400C002824D1012021
:1076C000CAE76068032809D15E48006801214906BD
:1076D0000840400E002817D10120BDE7606801284E
:1076E00008D15848006804210840800800280BD1C0
:1076F0000120B1E753480068012149020840400ACF
:10770000002801D10120A7E74E48C068800880000A
:10771000616808434B49C860FFF7E4FB06466068B0
:1077200002280FD107E0FFF7DDFB801B46498842A6
:1077300001D9032090E74348C0680C21084008287D
:10774000F1D134E0606803280FD107E0FFF7CAFBEE
:10775000801B3D49884201D903207DE73948C06834
:107760000C2108400C28F1D121E0606801280FD1DC
:1077700007E0FFF7B7FB801B3349884201D903209C
:107780006AE73048C0680C2108400428F1D10EE0B7
:1077900007E0FFF7A7FB801B2B49884201D9032094
:1077A0005AE72848C0680C2108400028F1D1244835
:1077B0000068C007C00FA8420ED9214800684008E1
:1077C000400028431E49086008460068C007C00FF3
:1077D000A84201D001203FE7042120680840042886
:1077E00008D11848C068072109028843E1680843A6
:1077F0001449C860082120680840082809D11148A8
:10780000C0680721C90288432169C90008430D499E
:10781000C86000F049F80B49C968F0221140090915
:107820000A4A515CC8400A4908600020FFF77EFB05
:107830000746002F01D038460EE700200CE7000075
:10784000002002400010024088130000AABC00087B
:10785000800100200148006870470000800100207E
:1078600000B5FFF7F7FF0549C9680722120211406A
:10787000090A034A515CC84000BD000000100240E4
:10788000BABC000800B5FFF7E5FF0549C968072243
:10789000D2021140C90A034A515CC84000BD000031
:1078A00000100240BABC0008FEB52E48C7680C2084
:1078B0003840002845D0042804D008280CD00C28D3
:1078C0003ED10BE02748006810210840002801D075
:1078D000254C00E0254C41E0254C3FE00F20800482
:1078E0003840800C23490E5C032080053840800D11
:1078F000401C01901B48C068012109040840002871
:1079000007D01B49714308460199FDF7F1FB054675
:1079100014E01448006810210840002807D01249DC
:10792000714308460199FDF7E3FB054606E00F4960
:10793000714308460199FDF7DBFB05462C460DE037
:1079400000BF08484068072149030840400B0090E9
:107950000098401C01218140CC0300BF00BF20469D
:10796000FEBD00000010024000093D000024F400AC
:1079700000127A00C2BC0008FEB50446002C01D1FA
:107980000120FEBDF848C6680C210E40C7680121E1
:1079900009040F402078C007C00F002872D0082EBD
:1079A00004D00C2E0FD1084687420CD1EE48006857
:1079B000012149040840400C002863D06068002879
:1079C00060D10120DDE700BF012109046068884221
:1079D00005D1E54800680843E349086027E0052130
:1079E0000904606888420ED1DF48006801218904DB
:1079F0000843DD490860084600680121090408437E
:107A0000D949086013E0D848006801210904884377
:107A1000D549086008460068012109040840009023
:107A200000BFD148006889008843CF49086000BF83
:107A30006068002813D0FFF755FA054606E0FFF707
:107A400051FA401B642801D903209AE7C648006810
:107A5000012149040840400C0028F0D012E0FFF753
:107A600041FA054606E0FFF73DFA401B642801D9BC
:107A7000032086E7BC480068012149040840400C07
:107A80000028F0D102212068084002287AD1E0685D
:107A90000290042E03D00C2E34D1002F32D1B248E4
:107AA0000068042108408008002804D002980028BB
:107AB00001D1012065E7AC4840681F2109028843D5
:107AC000216909020843A84948600846006809215D
:107AD000884302990843A4490860FFF7E5FEA249DC
:107AE000C968F02211400909A04A515CC840A04968
:107AF00008600020FFF71AFA01900198002841D091
:107B000001983EE70298002824D097480068092190
:107B100088430299084394490860FFF7E3F9054652
:107B200006E0FFF7DFF9401B022801D9032028E710
:107B30008D4800680421084080080028F1D08A4858
:107B400040681F21090288432169090208438649C8
:107B5000486017E084480068400840008249086097
:107B6000FFF7C0F9054606E0FFF7BCF9401B022805
:107B700001D9032005E77C480068042108408008FB
:107B80000028F1D1102120680840102867D1002E6C
:107B900036D17548006849010840400A002804D0E1
:107BA000A069002801D10120EBE66F484068072159
:107BB00049038843216A08436B4948600846406886
:107BC0000002000A217F0906084367494860206ACD
:107BD000400B401C01218140C8036349C968F02261
:107BE00011400909614A515CC840614908600020A0
:107BF000FFF79CF90190019800284BD00198C0E64E
:107C0000A06900282CD058480068FF2101310843A2
:107C100055490860FFF766F9054606E0FFF762F987
:107C2000401B022801D90320ABE64F480068012120
:107C300049020840400A0028F0D04B48406807211C
:107C400049038843216A0843474948600846406819
:107C50000002000A217F090608434349486019E0F1
:107C600041480068FF21013188433F490860FFF720
:107C700039F9054606E0FFF735F9401B022801D91E
:107C800003207EE638480068012149020840400A86
:107C90000028F0D1082120680840082839D16069FF
:107CA00000281BD0304840300069012108432E498C
:107CB00040310861FFF716F9054606E0FFF712F9B3
:107CC000401B022801D903205BE6274840300069A9
:107CD0000221084040080028F0D01AE02248403035
:107CE000006940084000204940310861FFF7FAF878
:107CF000054606E0FFF7F6F8401B022801D90320ED
:107D00003FE6194840300069022108404008002839
:107D1000F0D1042120680840042879D10020009087
:107D20001148806B89060840002806D10E48806BF8
:107D300008430D498863012000900E480068FF2128
:107D40000131084000281ED10A480068084309494B
:107D50000860FFF7C7F805460EE0FFF7C3F8401BC1
:107D6000642809D903200CE600100240AABC0008D0
:107D7000800100200070004085480068FF2101312B
:107D800008400028E9D000BFFF210131A0688842E7
:107D900005D18048006908437E49086130E0A06849
:107DA00000280DD17B480069FF21013188437949C2
:107DB00008610846006909158843764908611FE093
:107DC00005210902A06888420DD17248006901218D
:107DD000890208436F49086108460069891508430C
:107DE0006C4908610CE06B480069FF210131884350
:107DF00068490861084600690915884365490861B2
:107E000000BFA068002815D0FFF76CF8054608E011
:107E100031E0FFF767F8401B5F49884201D9032032
:107E2000AFE55C480069012149020840400A00288A
:107E3000EFD013E0FFF756F8054607E0FFF752F8DA
:107E4000401B5549884201D903209AE551480069F1
:107E5000012149020840400A0028EFD1009801287A
:107E600008D14C484038806B0121090788434949B3
:107E70004039886300BF606A00284CD00C2E69D05E
:107E8000606A022848D14348403800680121090649
:107E90008843404940390860FFF724F8054606E06A
:107EA000FFF720F8401B022801D9032069E5394873
:107EB00040380068012149060840400E0028EFD1F3
:107EC000E16AA06A0843216B084332494039C96816
:107ED000FD221204914308432E494039C8600846E8
:107EE00000680121090608432A4940390860FEF765
:107EF000F9FF054606E0FEF7F5FF401B022801D911
:107F000003203EE523484038006801214906084027
:107F1000400E0028EFD038E01E48403800680121AC
:107F2000090688431B4940390860FEF7DBFF054618
:107F300006E0FEF7D7FF401B022801D9032020E509
:107F4000144840380068012149060840400E0028C6
:107F5000EFD11AE0606A012800D112E50D484038DF
:107F6000C768012000043840A16A88420BD10F2065
:107F700080043840E16A884205D1032080053840FA
:107F8000216B884201D00120FBE40020F9E40000CD
:107F900000700040401002408813000010B50446F5
:107FA000002C01D1012010BD606A002800D100BF63
:107FB0000021A1625120005D002804D1502001550C
:107FC000204600F035F80221512001552068006854
:107FD0004021884321680860A16860680843E1681F
:107FE0000843216908436169084301225202A169DB
:107FF00011400843E1690843216A0843A16A084324
:1080000021680860A069000C04210840616A0843E7
:10801000216848602068C069910088432168C86170
:10802000002060650121512001550020BBE70000C0
:1080300010B586B00446142101A8FDF7CCF8144908
:108040002068884222D11348406B891408431149A3
:10805000486300BF0846C06A012108430D49C86251
:108060000846C06AC007C00F009000BF00BFE020F4
:108070000190022002900020039003200490002031
:10808000059001A905200007FEF726FE06B010BDE9
:10809000003001400010024070B504462546681EBD
:1080A0000949884201D901200CE0681E074948614E
:1080B0000321081F00F0A0FF002004498861072069
:1080C0000861002070BD0000FFFFFF0000E000E03D
:1080D00070477047FEB504462068C5692068066889
:1080E000206887682807000F0190019800280ED1AA
:1080F0002020284000280AD020203040002806D028
:10810000206E002802D02046216E8847FEBD0198CF
:1081100000287DD0F807C00F002804D1FF202130AF
:1081200030400028F5D0E807C00F00280BD0FF2012
:1081300001303040002806D0012021680862E06F3D
:1081400001210843E0670220284000280AD0F807F0
:10815000C00F002806D0022021680862E06F0421C9
:108160000843E0670420284000280AD0F807C00F21
:10817000002806D0042021680862E06F022108432D
:10818000E0670820284000280ED02020304000283A
:1081900003D1F807C00F002806D008202168086224
:1081A000E06F08210843E067E06F002846D02020F8
:1081B0002840002809D020203040002805D0206E1B
:1081C000002802D02046216E8847E06F009020688A
:1081D000806840210840402804D0082100980840C9
:1081E000002826D0204602F07CF8206880684021D4
:1081F0000840402819D12068806888432168886039
:10820000E06E00280DD02548E16E8863E06E00E046
:1082100015E0FEF737FB002810D0E06E816B884731
:108220000CE02046FFF755FF08E02046FFF751FF1E
:1082300004E02046FFF74DFF0020E06766E70120DD
:108240000005284000280CD0012080053840002877
:1082500007D001200005216808622046FFF738FF9B
:1082600054E78020284000280AD080203040002891
:1082700006D0606E002802D02046616E884745E730
:1082800040202840002807D040203040002803D05C
:10829000204602F038F839E700BF37E721A200088E
:1082A00010B50446002C01D1012010BDA0690028A2
:1082B00000D000E000BF606F002805D100217020D1
:1082C0000155204600F02CF82420606720680068E3
:1082D0004008400021680860204602F07BF8012831
:1082E00000D1E2E7606A002802D0204601F00AFED1
:1082F000206840680921C9028843216848602068D5
:1083000080682A21884321688860206800680121EC
:10831000084321680860204601F06CFEC5E70000B4
:1083200010B586B00446142101A8FCF754FF3E495D
:108330002068884275D13D48406B0121890308437C
:108340003A49486300BF0846C06A012108433749DB
:10835000C8620846C06AC007C00F009000BF00BFD7
:108360004815019002200290002003900320049001
:108370000420059001A905200007FEF7ADFC0120AF
:1083800080020190022002900120039003200490BB
:108390000420059001A905200007FEF79DFC244854
:1083A0002449086003204860002122488160C160A0
:1083B000802101610021416181612021C1610902A7
:1083C0000162FEF711FB002801D0FDF749FC00BF58
:1083D0001848E066846200BF1548143816490860E2
:1083E000032048601021144881600021C160802171
:1083F0000161002141618161C1610162FEF7F4FA0E
:10840000002801D0FDF72CFC00BF0B48A066846259
:1084100000BF002201211B20FEF7A6FF1B20FEF754
:1084200097FF06B010BD0000003801400010024068
:10843000300002405C170020A417002070B50446ED
:108440000D461646A06F202863D1002D01D0002EC6
:1084500001D1012070BD01210903A068884208D123
:108460002069002805D1E807C00F002801D00120AD
:10847000F0E700BF7020005D012801D10220E9E78C
:1084800001217020015500BF65655820065300206A
:10849000E0672220A067E06E002820D01E48E16E31
:1084A000C8621E48E16E08631D48E16E4863002003
:1084B000E16E88632368194624313346626DE06EAD
:1084C000FEF7E6FA00280AD01020E06700BF00217E
:1084D0007020015500BF202060670120BAE700BF6F
:1084E00000217020015500BF20680068FF21013184
:1084F00008432168086020688068012108432168DA
:1085000088602068806840210843216888600020D6
:10851000A0E702209EE700008BA20008D5A2000879
:1085200039A2000870477047FFB583B004460D4676
:108530001746606F202875D1002D01D0002F02D181
:10854000012007B0F0BD01210903A068884208D1CD
:108550002069002805D1E807C00F002801D00120BC
:10856000EFE700BF7020005D012801D10220E8E79D
:1085700001217020015500BF0020E06721206067C5
:10858000FEF7B0FC01905020075352200753012101
:108590000903A068884205D12069002802D100267D
:1085A000029502E02E460020029021E006980090FD
:1085B000002280212046019B02F0FAF8002801D019
:1085C0000320BEE7002E09D102980088C005C00D27
:1085D000216888620298801C029003E0307821684C
:1085E0008862761C5220005B401E81B252200153EB
:1085F0005220005B0028D9D106980090002240212B
:108600002046019B02F0D4F8002801D0032098E70F
:108610002020606700BF00217020015500BF0020AE
:108620008FE7FFE702208CE7704700BFFEE710B539
:108630000022042105200007FEF74DFC002208213E
:1086400005200007FEF747FC0A2002F039FC012252
:10865000042105200007FEF73EFC0A2002F030FC52
:108660000022042105200007FEF735FC10BD10B5DF
:108670000022042105200007FEF72DFC012208211D
:1086800005200007FEF727FC0A2002F019FC012252
:10869000042105200007FEF71EFC0A2002F010FC52
:1086A0000022042105200007FEF715FC10BD70B55F
:1086B0000546002400261EE00022042105200007B4
:1086C000FEF709FC0A2002F0FBFB01220421052031
:1086D0000007FEF700FC6006040E082105200007D5
:1086E000FEF7F0FB002801D0601CC4B2052002F0A8
:1086F000E7FB701CC6B2082EDEDB002D02D1FFF7AF
:10870000B6FF01E0FFF793FF204670BD70B5044649
:108710000022042105200007FEF7DDFB00252AE0EA
:1087200080202040C011002806D001220821052009
:108730000007FEF7D0FB05E0002208210520000716
:10874000FEF7C9FB6006040E0A2002F0B9FB012205
:10875000042105200007FEF7BEFB0A2002F0B0FB53
:108760000022042105200007FEF7B5FB0A2002F0D5
:10877000A7FB681CC5B2082DD2DB70BD10B5012265
:10878000082105200007FEF7A6FB01220421052091
:108790000007FEF7A0FB0022082105200007FEF7D6
:1087A0009AFB0A2002F08CFB00220421052000071E
:1087B000FEF791FB10BD10B5002204210520000733
:1087C000FEF789FB0022082105200007FEF783FB46
:1087D0000A2002F075FB0122042105200007FEF7A4
:1087E0007AFB0122082105200007FEF774FB0A200E
:1087F00002F066FB10BD10B50024012208210520FF
:108800000007FEF768FB062002F05AFB0122042154
:1088100005200007FEF75FFB062002F051FB07E092
:10882000601CC4B2FA2C03DDFFF7C5FF012010BDA8
:10883000082105200007FEF745FB0028F0D10022A3
:10884000042105200007FEF746FB0020EFE70000AB
:1088500038B501F007FC01F059FC5A480068C069BE
:1088600002210840002802D057485849C860FDF747
:1088700049FB044656480078002806D001280AD053
:10888000022819D0032824D11DE001229102514869
:10889000FEF721FB1DE0FF20F530844206DA0022BE
:1088A000012189024B48FEF716FB04E001229102E8
:1088B0004848FEF710FB0CE00022012189024548E0
:1088C000FEF709FB05E0012291024248FEF703FB97
:1088D00000BF00BF0121C9023E48FEF7F3FA00289D
:1088E0001CD03D48007863280BDD00220821394860
:1088F000FEF7F1FA0122D10305200007FEF7EBFA9B
:1089000018E0012208213348FEF7E5FA0022012190
:10891000C90305200007FEF7DEFA0BE0002208215C
:108920002C48FEF7D8FA00220121C90305200007D0
:10893000FEF7D1FA2948808C012820D1002528484B
:10894000009072B680212748FDF7A6F90546002D54
:1089500005D0022269462348FDF790FA054662B623
:1089600021A002F05BF800211C48818403F00CF97F
:10897000642002F09BFA14481449C86000BF1748ED
:10898000408C01280ED10021144841840020134955
:108990004039088003F0F8F8642002F087FA0A48AA
:1089A0000A49C8600D48008C01280AD100210B48F3
:1089B000018403F0E9F8642002F078FA02480349E0
:1089C000C86038BDDC1600200400FA0500ED00E0A8
:1089D000320100200004005048010020F40D002066
:1089E000AAAA0000384A0008BDF8C8EBC9FDBCB609
:1089F000C4A3CABD0D0A000008B53721202000F02D
:108A000077F80321212000F073F84021222000F0A4
:108A10006FF80821232000F06BF8AA21302000F025
:108A200067F802200B4908870846008FC1B2322040
:108A300000F05EF80121332000F05AF85F21202079
:108A400000F056F8684600F007F80A2002F038FAFD
:108A500008BD0000B40D002010B5044621460F20CB
:108A600000F023F8002800D110BD0120FCE770B50C
:108A700004460025FFF782FE3220FFF747FEFFF78E
:108A8000BAFEE0B2FFF742FEFFF7B5FEFFF776FE53
:108A90003320FFF73BFEFFF7AEFE0020FFF707FE97
:108AA0000546FFF788FE284670BD70B505460C46A2
:108AB0002846FFF7DCFF2070012070BD70B504462A
:108AC0000D46FFF75BFE3220FFF720FEFFF793FE17
:108AD000E0B2FFF71BFEFFF78EFE2846FFF716FEFB
:108AE000FFF789FEFFF767FE0A2002F0E9F970BD83
:108AF00070B504460D4629462046FFF7DFFF0120EA
:108B000070BD000010B50248FEF7B9FA10BD0000B4
:108B100054160020F0B585B004460020039072B6CC
:108B20004F4920684018002806D14E48C0680321EC
:108B300089040840039000E000BF00BF20688068FF
:108B400002902068C06801902068456920688669A5
:108B500043492068401800280DD142484038806AB7
:108B6000490508433F49403988620846806A400009
:108B70004008886200E000BF00BF002D01D1002E38
:108B80005FD0374920684018002807D13548C068B1
:108B90000321890488433349C86000E000BF00BF57
:108BA000002D1DD02068006901210843216808615B
:108BB00020684561FEF796F9074600BFFEF792F977
:108BC000C01B00902068006808210840082804D0D5
:108BD0007D21C90000988842F0D9082021684860AA
:108BE000002E1DD02068006901210843216808611A
:108BF00020688661FEF776F9074600BFFEF772F936
:108C0000C01B00902068006810210840102804D084
:108C10007D21C90000988842F0D910202168486061
:108C20000F4920684018002809D10E48C068032168
:108C300089048843039908430A49C86000E000BFDB
:108C400000BF206800694008400021680861029860
:108C50002168886001982168C86062B605B0F0BDDF
:108C60000084FFBF401002401CB50020009001901E
:108C70001E481F49086000211D48C163012080076C
:108C80001B49486000211A48816007218163012146
:108C900001610021C160001D01774177001F8162E1
:108CA000FF21C231416200212430017204212438A5
:108CB00041610021016381614163C161FDF7E2FB14
:108CC000002801D0FCF7CCFF0A48009080130190E7
:108CD00069460748FDF74AFB002801D0FCF7C0FFB2
:108CE00000210348FDF7D4FA1CBD00000024014018
:108CF000F81500200200000408B500BF0A48006B08
:108D000001210843084908630846006BC007C00FEB
:108D1000009000BF00BF002201210A20FEF724FBC3
:108D20000A20FEF715FB08BD0010024000B587B011
:108D3000142102A8FCF74FFA00BF6548C06A04215D
:108D400008436349C8620846C06A0421084001908C
:108D500000BF00BF00BF5E48C06A802108435C4975
:108D6000C8620846C06A80210840019000BF00BF69
:108D700000BF5748C06A012108435549C8620846E8
:108D8000C06AC007C00F019000BF00BF00BF084607
:108D9000C06A022108434E49C8620846C06A0221DF
:108DA0000840019000BF00BF01221C2105200007E0
:108DB000FEF791F8012247494748FEF78CF8002258
:108DC00046494548FEF787F800229121090205200F
:108DD0000007FEF780F80120029041480390002030
:108DE000049002A905200007FDF776FF02200290FB
:108DF000032003900020049002A905200007FDF73E
:108E00006BFF0C200290112003900020049003209F
:108E1000059002A905200007FDF75EFF10200290D3
:108E200001200390002004900220059002A9052053
:108E30000007FDF751FF0120029011200390002050
:108E40000490059002A92448FDF746FF02200290F5
:108E5000244803900120049002A91F48FDF73CFF1D
:108E6000214802900120039000200490059002A95F
:108E70001948FDF731FF0120C00202900020039045
:108E80000220049002A91448FDF726FF9120000259
:108E900002900120039000200490059002A9052073
:108EA0000007FDF719FF80200290002003900120A9
:108EB000049002A90848FDF70FFF002201210520B8
:108EC000FEF752FA0520FEF743FA07B000BD000096
:108ED00000100240010400000004005008300000AF
:108EE00000001110000021100834000010B50A48DD
:108EF0000A4908600020486000210848816008494C
:108F000041610021016241628162FEF743F900285C
:108F100001D0FCF7A5FE10BD007C004054160020D7
:108F2000FFFF000010B5124812490860FF2005300D
:108F3000486000210F488160C160016141610121E9
:108F4000490281610021C1610162416281620721A0
:108F5000C162FFF723F8002801D0FCF781FE054825
:108F6000006800684021084302490968086010BD94
:108F7000003001408416002000B585B014216846F9
:108F8000FCF729F919481A490860E12040024860B5
:108F9000002117488160C16001610C2141610021FD
:108FA0008161C161016230201149486201210903D8
:108FB0000F4881634900C163FFF772F9002801D0AF
:108FC000FCF74EFE0120800200900220019001205B
:108FD00002900320039004200490694605200007B6
:108FE000FDF77AFE01F026FC05B000BD0038014017
:108FF000DC1600207047000010B5002819DA1A4A64
:1090000003071B0F083B9B089B00D2588307DC0E0D
:10901000FF23A3409A438B071B0E8407E40EA34053
:109020001A43114B0407240F083CA408A4001A514A
:1090300018E00E4A03231B02D21883089B00D25863
:109040008307DC0EFF23A3409A438B071B0E840784
:10905000E40EA3401A43054B032424021B19840881
:10906000A4001A5110BD00001CED00E000E100E07A
:1090700000BF00BF00BFBFF34F8F00BF00BF00BFE6
:1090800006480749C86000BF00BF00BFBFF34F8F4D
:1090900000BF00BF00BF00BF00BFFDE70400FA052E
:1090A00000ED00E0F0B593B000200E90962002F0A5
:1090B0007FFA4B20C00002F097FA0020FE490870AA
:1090C000FE4800780C2802DB0B20FC4908700122C6
:1090D000510205200007FDF7FEFEF8480078F84928
:1090E0000870F6480078F74908700020F6490870C3
:1090F000F6490870F6480078F64908710221F648EA
:10910000FDF7E0FE002801D1012000E00020F14938
:10911000C871F24801780068401CF04A1060C8B27B
:10912000EC49C870E74800788872E6480078420049
:10913000EB49E8480B30FCF735F80620E549487262
:109140000846E8490A78427049788170DD49097813
:10915000490008460D300022DE4902F047FBD9499C
:109160000978490008460D30002102F053FB022027
:1091700002F078FA0020DC4908700120DB49087011
:109180000020DB490870DB48FEF790F8DA490880D8
:109190000020CD490870CB480078FCF75DFA064600
:1091A000FCF7DAFAD54AD64B05910490FCF774F92E
:1091B0000791069001F016FE002201239B070991FA
:1091C0000890FCF7B7F80B910A90FCF7A7FAC0B229
:1091D0000D900D984001C84909884018C949088078
:1091E000084600880121C903884204DBC54800887D
:1091F000401AC4490880C448C4490860C44800787B
:10920000401CC3490870BB48FEF750F8C1490880AC
:109210009DE2B848FEF74AF8BE49088033E0B248FC
:10922000007800281BD002F07FF910901299109856
:10923000884214D911991098884210D201F0F2FF97
:109240000020AA490870384602F0AAF9012002F06D
:1092500009FAB14908700020A34908701DE0A5482B
:10926000FEF724F8AB49088008460088A54909881C
:10927000884208DBA7480088A2490988A74A8918BC
:10928000884200DA09E000210F2002F0E9F8A44941
:109290000860A44908400028C1D000BFA048006869
:1092A000401C002801D1FFF7E3FE9D480068012122
:1092B0008903084000287DD08122D20100210F209F
:1092C00002F04DFA0021102002F0CAF84006400ECC
:1092D0000F90002294480F9902F012F9002002F03A
:1092E00083F9002002F02FF98F48407A07288FD1A8
:1092F00002228E498C48401DFBF778FF002887D159
:1093000002F0E5FA8A4A03C202F0CAFA894A03C2A5
:109310006D480078401C6C4908708348427808A961
:109320000A748078487466480078002810D10120BB
:10933000814908706846008E6949088001206149AA
:109340000870644908A8007C487008A8407C8870B0
:10935000634800886946098E88427DD17749724802
:10936000C089088076487049098A01806148FDF704
:109370009DFF6849088072480088FF30C3307049FB
:109380000880084600886F49884212DD6C480088D2
:10939000401A6B49088069480088401C674908806A
:1093A0000846008867490B31884202DB0020634988
:1093B000088000E0BFE10026032063498855634927
:1093C000594842890A808089488008460068B1006F
:1093D0005F4A50505448C07C0007000F032805D056
:1093E0005148C07C0007000F384908704E48C07CC7
:1093F00000115849087000204549087001203A4979
:1094000008704249484842890A80808948802D482E
:109410000078FF2191314843FF309B30FF30F53019
:109420000004C117434B0CCB801859410906070AA9
:109430000F434948381A12901920800238181190A9
:109440007908490000200A0E000210430B02002296
:1094500011469A18484100E00EE140490A60486010
:1094600033480CC81B480A3002F000FA31480CC8D7
:109470001848163002F0FAF938480CC8154812306E
:1094800002F0F4F90820134948720E49097889005E
:1094900008461C3000220F4902F0A8F90949097852
:1094A000890008461C30002102F0B4F9012010495F
:1094B000087004221C4953E0E90000202A01002022
:1094C000290100202801002009010020320100208C
:1094D0004801002028120020000400506C000020E9
:1094E00022140020020100201C0100201E01002087
:1094F0001D01002054160020220100209A999999FC
:109500009999D93F24010020A08601000401002080
:109510001901002020010020E8000020983A0000F6
:109520007000002000D02724781200203C01002089
:1095300078000020800000201B0100204401002052
:10954000F4000020E7030000E4140020F8000020ED
:109550005414002033010020005203008800002032
:10956000491CF948FBF71EFEF84800887D21C90018
:109570004843F74909884018F6490860F6480078DA
:10958000F6490870F649C888FCF766F80990EF4874
:109590000088FCF761F808900999FBF78DFE7F21A0
:1095A000C9050A90FBF72FFE0B90FCF77FF8EA49FC
:1095B0000880EA480078401E0988884202D10120CC
:1095C000E8490870E1480088E7490880E749002039
:1095D000085EFCF749F809910890E5480088FCF717
:1095E00057F8E44AE44B01910090FBF755FF0591D1
:1095F0000490D8480068FCF737F803910290059B67
:10960000049AFBF73BFF07910690099B089AFBF72A
:1096100091FE0B910A90FCF75DF8D8490860D84894
:10962000008800F057FBD748007800287ED0CC484F
:1096300040300088D349097888427BD0D1480178EE
:10964000C748403001801222CF49D048FBF7AAFD1D
:109650000822CE49C248801DFBF7A4FD0A22CB494F
:109660000831BF483630FBF79DFD02F08DFA6420CB
:1096700001F01CFCFFF7FCFC6846008EFCF72CFC9C
:109680000646C34909788E4213DB0120C1490870A0
:10969000C1480078401CC04908706846008E7100BF
:1096A000BE4A5052BE4908A8007C487008A8407CB9
:1096B00088700320BB498855BB49B3481438428998
:1096C0000A808089488008460068B100B74A505037
:1096D000AD481438C07C0007000FB54909788842AE
:1096E0000BDDA9481438C07C0007000F032804D004
:1096F000A5481438C07CAE490870B0001630A8499F
:1097000040180B90AB480CC80B9802F0AFF8A24978
:109710000978890008461C300022A14902F066F849
:109720009D490978890008461C3000E002E00021CC
:1097300002F070F80BE0A04A00210F2002F00FF8B1
:109740009E480078002802D0002001F0FCFE8848E6
:1097500000889B490988884200DA5AE584480088D5
:1097600097490988974A89188842F6DC924A00216D
:109770000F2001F0F4FF9448007887490870002515
:1097800088480078002818D16F480068FCF790FCE2
:109790008E49088008880988491E8C4B19808C499D
:1097A0000988FBF7BBFC8B480088414388B27449A9
:1097B00008800846008800F08DFA0020864908706D
:1097C000002423E07748005D00281DDD82480078F2
:1097D000401C814908707348005DA9007F4A5050C1
:1097E00060006E49085A69007D4A5052A0006F49D6
:1097F0000A582846691CCDB280007A490A50694847
:10980000005D401E67490855601CC4B2604800787E
:10981000604909784018A042D4DC6B4800780328DE
:1098200003DA6D4800786C4908706B480078584935
:10983000087000243FE0002536E0A8006949095877
:10984000681C8000674A105881422BDDAA00654BD6
:1098500099586A00624B985AA200604B9A580C9231
:109860006A1C92005F4B9A58AB005E4EF2506A1C25
:1098700052005B4B9A5A6B00594EF2526A1C92008E
:10988000564B9A58AB00554EF2506A1C9200554BFD
:1098900099506A1C5200524B98526B1C9B000C9AB8
:1098A000F25000BF681CC5B239480078401EA8427B
:1098B000C3DC601CC4B236480078401EA042BADC4B
:1098C000002049490870002438E060004449085AE3
:1098D0006100324A5052A00042490858A100334A60
:1098E0005050A000114608584049884224D0A0009A
:1098F0003A4908580A281FD13B48007806214843B6
:10990000001D3B4940186100244A89180A780270FA
:1099100049784170A200254BD118334A12780623AA
:109920005A43921D324BD0180422FBF73BFC2E48C1
:109930000078401C2C490870601CC4B214480078A0
:109940008442C2DB00245BE02C01002044010020A3
:10995000F40000200C010020620100202B010020F7
:10996000B40D00201D010020260100203001002040
:1099700020010020F853E3A59B843E401401002001
:109980004A010020330100208C120020F014002036
:10999000290100201B0100202801002022140020A2
:1099A00028120020E4140020F800002054140020A5
:1099B000320100208000002000D027241E0100205A
:1099C00024010020983A000009010020FC0000203A
:1099D000500100204E0100202A010020B414002074
:1099E0003A140020841400201A010020FFFF010017
:1099F000D61300200A48A1000A4A5050601CC4B285
:109A00000C2CF7DB084A00210F2001F0A8FE0022F1
:109A10000121490205200007FDF75DFA13B0F0BDF2
:109A2000FFFF01005414002080D02724704700005D
:109A3000F0B585B048484949086002F031F8FF2088
:109A40001030474948800846C08E4649087044484F
:109A5000C08F454908704248808F4449087040488B
:109A6000807A434908703E488088424908603C49F2
:109A70000889FBF70DFE04463F4A404BFBF70CFDFF
:109A80000191009001F0AEF90646002201239B07E8
:109A9000FBF750FC03910290FBF740FE3849088029
:109AA0002F49C88836490988FBF738FB35490880B3
:109AB0002B49888833490988FBF730FB30480088F8
:109AC000414388B23049088009887D22D200514341
:109AD0000846FBF7C9FD06462C4A2D4BFBF744FD13
:109AE0000446FBF71BFE2B490880274800882A49BB
:109AF00008801B48C1887D20C000FBF70FFB274969
:109B000008801748C1887D20C000FBF707FB244967
:109B10000880012023490880FCF7F4F922490880D5
:109B20001C48028821492248FDF7C4FB002801D0C7
:109B3000FCF796F80F4801681EA000F06FFF084878
:109B4000C18820A000F06AFF0548018922A000F02A
:109B500065FF05B0F0BD000041A8000848000020E6
:109B6000B40D0020010000205E0100205F010020F4
:109B7000470100203C0100209A9999999999D93F71
:109B80004E010020500100204A010020F853E3A5B7
:109B90009B843E40560100205A01002058010020BD
:109BA00060010020620100205C010020FF7F0000B6
:109BB00054160020B1EAC7A949443A202564202E52
:109BC0000D0A0000CDA8D1B6BCE4B8F43A20256453
:109BD000206D732E0D0A0000B5A5B4CECDA8D1B668
:109BE000BBF9D5BECAFDC1BF3A202564B8F62E0D1B
:109BF0000A00000000B585B014216846FBF7EBFAB7
:109C000000220121C9031048FDF765F90120C003B6
:109C100000900120019000200290039069460A48BC
:109C2000FDF75AF80120C0030090032001900020A6
:109C30000290039069460448FDF74EF8022001F0B7
:109C400035F905B000BD0000000400507047000069
:109C500038B504460D460020009055201B49087079
:109C6000AA20487003208870601DC8700320087106
:109C70000846457184716800154A811822461348C8
:109C8000C01DFBF78FFA002008E0811C0F4A525CD0
:109C90006946098851188AB20092401C611D8842A9
:109CA000F3DB0A48801CFBF729FF0090E01D074901
:109CB0004118684600780870684640784870214628
:109CC0000931024800F038FB38BD00009215002031
:109CD000B40D0020F0B585B005461A4800881A4931
:109CE0000988884206DB1748008817490988401A06
:109CF000144908801548C088124909884843471903
:109D00007D21C9004F43124800683E1A3046FBF7D8
:109D1000ABFC104A104B01910090FBF725FC03911E
:109D20000290FBF7D7FC04460C498C4201DD084643
:109D3000241A002C01DA09482418094800684461F3
:109D400005B0F0BD6201002060010020B40D0020CC
:109D500014010020F853E3A59B843E40FF7F0000E0
:109D60005416002001460020054A126890B2054AA8
:109D7000104002460A431046014A10607047000036
:109D800000300140C7FF000010B5FDF7B1F810BD6D
:109D900000B599B034210CA8FBF71DFA142107A8CF
:109DA000FBF719FA1C216846FBF715FA24480068EE
:109DB0000321C90288430121C902401820490860D3
:109DC000FDF7E4FA1F4800690321C90288431D49D1
:109DD000086106200C9088150E9001200F9010202D
:109DE0001090022015900021169141041791410511
:109DF00018910CA8FDF7C0FD002801D0FBF730FF3B
:109E00000F20079003200890002009900A900B90E3
:109E1000012107A8FDF71AFC002801D0FBF720FF5D
:109E20008120009000200290032080040690684664
:109E3000FDF7F6FA002801D0FBF712FF19B000BDBC
:109E4000007000404010024015480068FF210131B9
:109E50000843134908600846C06812490840104981
:109E6000C86008460068104908400D490860084667
:109E70008068400840008860084600680121890425
:109E80008843074908600846C068FD2109048843E3
:109E90000349C8600020086104480549886070478C
:109EA000001002400C40FF88F6FFF6FE005000084C
:109EB00000ED00E010B501F0EDFA044602E001F01B
:109EC000E9FA04460C488442F9D100200B49088085
:109ED0000B480078002804D0012803D0022807D1BD
:109EE00003E005E0FCF730F802E0FFF7DBF800BF25
:109EF00000BF01F07BF910BD3001CADEE600002092
:109F000060000020818CC907C90F002908D00168B2
:109F10004968012252049143826A114302685160E8
:109F20000222416A1140022907D101684968D2031F
:109F30009143C26A1143026851600422416A114090
:109F4000042907D10168496812049143026B114347
:109F5000026851600822416A1140082907D101684E
:109F6000496812039143426B114302685160102209
:109F7000416A1140102907D1016889681202914392
:109F8000826B1143026891602022416A11402029AE
:109F900007D10168896812029143C26B11430268BC
:109FA00091604022416A1140402915D101684968F9
:109FB00092039143026C1143026851600122120521
:109FC000016C914208D1016849680322520591430E
:109FD000426C1143026851608022416A114080291D
:109FE00007D10168496812039143826C11430268EA
:109FF0005160704738B504460020E067FCF772FFF7
:10A000000546206800680821084008280BD114483C
:10A010002B46002289040090204600F0C9FB00284E
:10A0200001D0032038BD20680068042108400428BE
:10A030000BD10B482B46002209050090204600F06A
:10A04000B7FB002801D00320ECE720206067A06761
:10A0500000BF00217020015500BF0020E2E7000092
:10A06000FFFFFF0170B50025C824204800780028B4
:10A0700000D070BD1E480078002800D0F9E701200C
:10A080001B4908701B48406B002801D10870F0E79D
:10A090001848406BC8210D1A1CE01749174A12686E
:10A0A000885C174909688847164800880A21484390
:10A0B0001549088011480068401C1049086008468E
:10A0C0000068C82801DB002008600A48406BC821EE
:10A0D0000D1A641E09480068A84201D0002CDCDC7F
:10A0E00000200349087000BFC3E7000042000020C1
:10A0F0004400002000000240EC0C0020380000204A
:10A1000048000020580100206801002010B53A489E
:10A110000078002803D139480078002800D010BD0D
:10A120000120364908703648C0698021084000285F
:10A1300002D132490870F2E732490020085632490C
:10A1400000228A56904215D12D48C069402108400E
:10A1500000280BD02D480078002807D000202B497C
:10A1600008702B480088401C29490880002023499A
:10A170000870D4E725480078002805D1012023493C
:10A1800008700A2000F09CFE1F4900200856CC21D0
:10A19000484320494018001D1F490968405C184980
:10A1A00088621D480068401C1B4908601649002051
:10A1B0000856CC214843174908581749096888426E
:10A1C00014DC0020144908600F480078401C40B29D
:10A1D0000D490870084600780E2801D1002008704B
:10A1E0000E480078401C40B20C490870002003491A
:10A1F000087000BF93E700004200002043000020E9
:10A2000000380140350000203400002045000020C7
:10A2100052000020C4010020580000203600002019
:10A2200070B50546AC6A00215A20015352200153F3
:10A230002046FDF74EFF70BDF8B50546AC6A666F67
:10A24000A76F2068806880210840802807D1212ED0
:10A2500005D1002152200153204600F064F8206807
:10A26000806840210840402807D1222F05D10021D5
:10A270005A200153204600F034F8E06F10210843C3
:10A28000E0672046FDF725FFF8BD70B50546AC6ACE
:10A290002868006820210840002817D100215A2092
:10A2A000015320680068FF2101318843216808605C
:10A2B00020688068400840002168886020688068C5
:10A2C00040218843216888602020A0672046FEF74F
:10A2D00029F970BD70B50446A56A2846FEF723F932
:10A2E00070BD01680968FF22213291430268116044
:10A2F00001688968490849000268916020218167E6
:10A3000000210166704710B50446206800684021AE
:10A31000884321680860202060670020606620462E
:10A32000FEF782F910BD01680968C02291430268F6
:10A33000116020214167704770B505460C462048E2
:10A340000078002803D11F480078002800D070BD95
:10A3500001201B490870C82C04DC1B480021415611
:10A36000002903DC002016490870F0E71749002097
:10A370000856CC21484316490C50144A0021515626
:10A38000CC225143124A8918081D22462946FAF761
:10A3900009FF0E480078401C40B20C49087008467E
:10A3A00000780E2801D10020087007480078401E70
:10A3B00040B20549087000200149087000BFC6E797
:10A3C000420000204300002036000020350000201D
:10A3D000C4010020F0B587B0044610200490002589
:10A3E000002003900026E7492068884200D100E061
:10A3F00000BF2169A068084361690843E169084317
:10A40000074620680068E049084038432168086032
:10A4100020684068032109038843E16808432168F4
:10A420004860A769D7492068884201D0206A07435D
:10A43000206880680B2109028843384321688860BE
:10A4400000BFD249206888421CD1D148C06880072B
:10A45000800F002806D001280AD0022805D0032842
:10A460000CD108E0012004900BE00220049008E0E9
:10A470000420049005E00820049002E010200490DD
:10A4800000BF46E0C349206888421CD1C048C0686C
:10A490000C210840002806D004280AD0082805D03E
:10A4A0000C280CD108E0002004900BE0022004905E
:10A4B00008E00420049005E00820049002E0102049
:10A4C000049000BF25E0AF49206888421FD1B04802
:10A4D000C068032189020840002808D001218902B0
:10A4E000401A0AD0401A05D0401A0CD108E00020CA
:10A4F00004900BE00220049008E00420049005E0A2
:10A500000820049002E01020049000BF01E0102019
:10A51000049000BF9B492068884256D104980428C3
:10A520001AD004DC002807D002281CD108E0082833
:10A5300016D0102817D117E0FDF792F9064616E05D
:10A54000934840380068102108400009002801D0D5
:10A55000914E00E0914E0AE0FDF7A6F9064606E0AE
:10A560000126F60303E000BF0120039000BF00BFF7
:10A57000002E0AD0606841004018B04203D86068DD
:10A580000003B04202D201200390F4E06068029020
:10A590003046FF21013100F068FA6268520800235A
:10A5A0008018594101910090029AFAF7CBFD0546B7
:10A5B00003200002854205D37948854202D82068ED
:10A5C000C560D8E001200390D5E00121C903E0690E
:10A5D00088426FD1049804283CD006DC002809D0BA
:10A5E000012813D002284AD11CE008283ED01028A8
:10A5F00045D145E0FDF734F940006168490840184D
:10A6000002906168FAF774FD85B23CE0FDF73AF913
:10A61000400061684908401802906168FAF768FDD7
:10A6200085B230E05A4840380068102108400009DF
:10A63000002807D061684A085A4BD018FAF758FD2D
:10A6400085B206E061684A08574BD018FAF750FD0A
:10A6500085B218E0FDF728F9400061684908401804
:10A6600002906168FAF744FD85B20CE061684A081F
:10A6700001231B04D018FAF73BFD85B203E000BFAD
:10A680000120039000BF00BF102D0FD34748854223
:10A690000CD846480F38284005902807400F0599E8
:10A6A0000843059005982168C86064E00120039084
:10A6B00061E0FFE7049804283AD006DC002809D0BE
:10A6C000012812D0022847D11AE008283BD01028D0
:10A6D00042D142E0FDF7C4F8616849084018029091
:10A6E0006168FAF705FD85B23AE0FDF7CBF86168DD
:10A6F0004908401802906168FAF7FAFC85B22FE029
:10A70000234840380068102108400009002807D07D
:10A7100061684A08204BD018FAF7EAFC85B206E0D7
:10A7200061684A081D4BD018FAF7E2FC85B217E0C1
:10A73000FDF7BAF861684908401802906168FAF7B5
:10A74000D7FC85B20CE061684A080123DB03D0180E
:10A75000FAF7CEFC85B203E000BF0120039000BFF2
:10A7600000BF102D05D31148854202D82068C5606E
:10A7700001E001200390002020666066039807B086
:10A78000F0BD000000480040F369FFEF00380140D1
:10A79000401002400044004000093D000024F40045
:10A7A000FFFF0F0000127A000048E801FFFF0000E1
:10A7B000FFB581B004460D4617460A9E22E0701C84
:10A7C00000281FD0FCF78EFB0499401AB04201D834
:10A7D000002E17D120680068FF21A131884321682D
:10A7E0000860206880684008400021688860202058
:10A7F0006067A06700BF00217020015500BF0320E3
:10A8000005B0F0BD2068C0692840A84201D10120F0
:10A8100000E00020B842D2D00020F1E710B51020AF
:10A820000349096808620248FDF754FC10BD0000A6
:10A83000DC1600200D20014908707047360000200A
:10A8400070B5044600256A480078082865D100BF25
:10A85000002004E06749095C49198DB2401C664933
:10A860000978491F8142F5DC64480078281885B2D0
:10A8700061480078281885B261480078281885B2A8
:10A8800060480078281885B25F480078281885B29B
:10A890006019C007C00F002835D05848007801283B
:10A8A00027D002282DD15949554A12788818554980
:10A8B0000A785049FAF776FC01F066F9642000F056
:10A8C000F5FA00BF00BF00BF00BF00BFBFF34F8F4E
:10A8D00000BF00BF00BF4E484E49C86000BF00BF68
:10A8E00000BFBFF34F8F00BF00BF00BF00BF00BF5E
:10A8F000FDE743480078411042480078FFF7A8F987
:10A9000000E000BF00BF0020394908703C490870D2
:10A91000394908704049087068E0354800780728D0
:10A9200012D134483C49097844543B480078401CD3
:10A930003949087030480078401F0978884255D15D
:10A9400008202B49087051E029480078062805D1D5
:10A950002C48047007202649087047E024480078F6
:10A96000052805D1264804700620214908703DE0DD
:10A970001F480078042805D12048047005201C4990
:10A98000087033E01A480078032808D11A48047088
:10A9900000201B49087004201549087026E014485F
:10A9A0000078002805D1552C03D1012010490870EA
:10A9B0001CE00F480078012805D1AA2C03D1022001
:10A9C0000B49087012E00A480078022807D1032CCE
:10A9D00005D10320064908700B48047006E00020EA
:10A9E00003490870064908700349087070BD0000EB
:10A9F000350100202E150020370100203A010020EB
:10AA0000380100203601002039010020B40D00205B
:10AA10000400FA0500ED00E03B0100200FB410B582
:10AA200003A9044B044A029800F034F910BC08BC96
:10AA300004B0184789B80008840100202021020CC6
:10AA400001D010211046020A01D01046083902092F
:10AA500001D01046091F820801D01046891E420805
:10AA600001D0881E7047081A7047F8B582B28BB2C1
:10AA7000040C0D0C10465843002126465E43370C4B
:10AA800036048019794116466E43370C3604801916
:10AA9000794126466E438919F8BD30B47446641E68
:10AAA0002578641CAB4204D3635D5B00E31830BCC3
:10AAB00018471D46F8E702E008C8121F08C1002A1F
:10AAC000FAD170477047002001E001C1121F002A2F
:10AAD000FBD1704708B5002100916B46012202218D
:10AAE0002C2000F051FE022100916B4601222C2007
:10AAF00000F04AFE08BD000038B504466D20009005
:10AB00006B46012208492E2000F03EFE002C05D0A5
:10AB1000064A07492E2000F011FE04E0054A0449C8
:10AB20002E2000F00BFE38BD0608000007060000CE
:10AB3000061800000716000038B504466B460222CE
:10AB40000021362000F0ACFC2300FFF7A6FF0E1119
:10AB5000081A54545454233154543D444B54002146
:10AB6000684601704078FE2108406946487043E01D
:10AB700069460878FC2108400121084369460870AD
:10AB80003AE069460878FC210840022108436946FA
:10AB9000087031E068460078B3210840482101433D
:10ABA000684601704078802108436946487023E078
:10ABB00068460178B320014068460170407841063C
:10ABC000490E6846417017E06946487802210843FB
:10ABD0006946487010E069464878FD21084069469A
:10ABE000487009E069460878CF21084020210843D1
:10ABF0006946087000E000BF00BF6B4601220021DB
:10AC0000362000F0C1FD00AB013301221146362091
:10AC100000F0BAFD38BD08B5032168464170012136
:10AC200001706B4602220021362000F0ADFD0122AA
:10AC3000D20306212D2000F081FD012000F036F91D
:10AC40000120FFF779FF08BD38B504462004010E46
:10AC50006846417004706B46022204212D2000F0EA
:10AC600093FD0321684601706B46012206212D20C9
:10AC700000F08AFD0021684601706B460122062122
:10AC80002D2000F081FD0A212D2000F0E9FB054672
:10AC9000284638BDFFB58DB00446002506E02528BE
:10ACA0000AD0109A0F999047641C6D1C20780028D8
:10ACB000F5D1284611B0F0BD00270121484A009780
:10ACC00000E00743641C23780846203B984010426C
:10ACD000F7D120782E2817D1042007436078641C10
:10ACE0002A280CD10E98641C02C800910E900BE02B
:10ACF00000990A22514330394018641C0090207892
:10AD0000014630390929F3D920780028D1D06428A8
:10AD100008D0692806D075281ED0109A0F99904740
:10AD20006D1C5BE00A200E99019001C90E9100286C
:10AD300002DA40422D2102E0390504D52B216A4672
:10AD40001172012103E0F90704D02021F7E70BAECF
:10AD50000B910DE00021FAE70A200E99019001C93C
:10AD60000E91F7E70199FAF7C3F93031761E317089
:10AD70000028F7D103A8801B20300190780701D567
:10AD8000009801E0012000900199884201DD401AFD
:10AD900000E000200027009006E002A8109AC05DA5
:10ADA0000F9990476D1C7F1C0B988742F5DB04E0E0
:10ADB000109A30200F9990476D1C0099481E009002
:10ADC0000029F5DC05E03078109A761C0F99904741
:10ADD0006D1C0199481E01900029F4DC641C65E794
:10ADE00009280100F8B54A002B4B520DD6182B4A02
:10ADF0000C460546142E2BDA002E12DA284BFAF7F1
:10AE000099FA00221346FAF7BBFC40D2002C03DA71
:10AE10000124E40700253AE02046284337D0214C9E
:10AE200014E0214F0B46F7403B402B4331D01C4BE5
:10AE3000FAF780FA00221346FAF7A2FC27D2002C78
:10AE400003DD01200005F0400419BC4300251EE08D
:10AE5000332E1EDC33460027143BFF43DF403842CD
:10AE600017D00F4BFAF710FB00221346FAF788FCB5
:10AE70000DD2002C0ADD142E0CD03420811B0120B1
:10AE800088404019A84200D2641C0546BD432146B3
:10AE90002846F8BD641CF9E701FCFFFF9C7500889B
:10AEA0003CE4377E0000F03FFFFF0F0070B5044622
:10AEB0007D20C00060430546284600F001F870BDC3
:10AEC000002100BF40E000BF00BF00BF00BF00BFC7
:10AED00000BF00BF00BF00BF00BF00BF00BF00BF7A
:10AEE00000BF00BF00BF00BF00BF00BF00BF00BF6A
:10AEF00000BF00BF00BF00BF00BF00BF00BF00BF5A
:10AF000000BF00BF00BF00BF00BF00BF00BF00BF49
:10AF100000BF00BF00BF00BF00BF00BF00BF00BF39
:10AF200000BF00BF00BF00BF00BF00BF00BF00BF29
:10AF300000BF00BF00BF00BF00BF00BF00BF00BF19
:10AF400000BF00BF00BF491C8142BCD37047000056
:10AF5000F0B585B004460020049003902578607910
:10AF600040008A49085A02906078401E8849C6B25B
:10AF70000863042D01D0072D01D1012000E000203D
:10AF80000190207882490873E07900280AD10846A8
:10AF900080690121890508437D4988610298C010B4
:10AFA000029006E07A488069012189058843784942
:10AFB0008861207A7649487308468069217A0904B5
:10AFC0000322120411400843714988610846002198
:10AFD0008269042000F0C3FB6E492E20029A00F023
:10AFE000ADFB3046FFF788FD6B48405D810040189F
:10AFF0006A494318052207212B2000F0C5FB684948
:10B0000001980B1801220B21282000F0BDFB62489B
:10B01000405D800063490A580C21282000F09FFB06
:10B02000E079800060494018A1794900425A022124
:10B03000272000F083FB70005C490A5A0421272076
:10B0400000F07CFBE079002805D16422062127204E
:10B0500000F074FB1EE0A07804280DD110200090B1
:10B0600010220621272000F069FB6B4601222621D1
:10B07000272000F089FB0DE02820009020220621E7
:10B08000272000F05BFB6B4601222621272000F0E1
:10B090007BFB00BF300146494018E17889004258E7
:10B0A0000821272000F05BFBA17A627A0802104396
:10B0B000002803D13F496172090AA172A17A637A1B
:10B0C0000802184302462021272000F037FB3A48A7
:10B0D0000C210268232000F042FB71003648001D5D
:10B0E000425A0421232000F029FBA07900280BD02C
:10B0F000E0793249431801220021212000F044FB6D
:10B1000003200490012003902807000F2901F0225A
:10B1100011400843617889040322920411400843D6
:10B12000049909059200114008430399490401223A
:10B13000520411400843217989051F2292051140CC
:10B1400008436179C906C90EC906084307463A464D
:10B1500000211F2000F003FBA07861780843000461
:10B160000B49086108460069E17949030122D203CD
:10B170001143084306490861084600210269082076
:10B1800000F0EDFA002005B0F0BD000078BC00082A
:10B19000880100200428000020BC000802000020D4
:10B1A0002000002028BC000848BC000854BC00084F
:10B1B00058BC00084110000040BC000822000020DC
:10B1C00038B504460D460848808B044322460021CA
:10B1D0002C2000F0B3FA00956B46012206212C20AA
:10B1E00000F0D2FA38BD00008801002010B5FFF74A
:10B1F00071FC10BD70B505460421362000F030F911
:10B200000446002D03D00120C002044304E00121C4
:10B21000C90220468843044622460421362000F015
:10B220009EFA70BD38B54020009000210E2000F03D
:10B2300017F90446002211460E2000F090FA6B46E2
:10B24000012200210D2000F09FFA084A00210F2062
:10B2500000F085FA00F056FA224600210E2000F098
:10B260007EFA00210248017338BD0000F8FF272450
:10B27000A8010020F0B585B0064604200290002702
:10B280000020019066494875086300216448203019
:10B29000417101730020624988834863886300F02C
:10B2A000F9F85F49086003E000F0F4F85C490860D1
:10B2B0005B4800685B498842F6D10020FFF73CFC00
:10B2C00059480078432802DD432057490870564802
:10B2D0000078002802DA00205349087052480078AC
:10B2E000242804DD504800780446243C0DE0062163
:10B2F0004D480078F9F712FF0621081A45014A481F
:10B300000078F9F70BFF2C460C4320062104084374
:10B31000210208432043039000211E20039A00F0DD
:10B320001EFA02AB01220021242000F02DFA1E207B
:10B33000FFF78AFC87B23812394988730420FFF777
:10B3400083FC01900198C0B200280FD00220009029
:10B350006B46012212212D2000F016FA3048808B16
:10B360000121090308432E49888300BF00F092F8A9
:10B370002B4908600620FFF767FC29494860072031
:10B38000FFF762FC26498860F806C00E087508467B
:10B39000007D002801D1102008752149087D00F0AA
:10B3A0004BFAF007C00F002809D0FFF734FC1C4807
:10B3B000808B0121C9020843194988830CE00521CB
:10B3C000362000F035F80546184805402A46052184
:10B3D000362000F0B3F900BF0120FFF7ADFB0021DC
:10B3E000042000F03DF80E4988610021262000F07D
:10B3F00037F80546052080030543800005432A46AB
:10B400000021262000F0ABF900222621362000F092
:10B4100095F900F03FF802490860002005B0F0BD42
:10B42000880100203001CADE01000020FFFD00007D
:10B43000F8B504460D46094FA9B2A0B26B460222E8
:10B4400000F02EF80646002E06D16846407801022C
:10B4500068460078081887B23846F8BDFFFF00003C
:10B46000FEB505460E460027FF43B1B2A8B201ABB8
:10B47000042200F015F800900098002808D1032459
:10B4800004E0380201A9095D4718641E002CF8DAAF
:10B490003846FEBD10B500210846FFF7E1FF10BD9C
:10B4A000FFB581B006460C4617460025002C04D196
:10B4B00029466D1C684646541AE040203043C2B20B
:10B4C00029466D1C684642547F2C04DC28466D1CBE
:10B4D00069460C540CE0E0B28021084329466D1CFB
:10B4E0006A4650546004020E28466D1C69460A5490
:10B4F000A8B23A466946049B00F012FB05B0F0BDC5
:10B5000070B504460D46164623462A46314611209C
:10B51000FFF7C6FF70BD10B5044623460522002183
:10B520001520FFF7BDFF10BD10B501210620FFF764
:10B5300097FF10BD10B504462346052200211720B1
:10B54000FFF7AEFF10BD38B504460020009000F0B4
:10B55000D9F8FF250135002C01D0680005432A46A3
:10B5600000210D2000F0EAF8002C17D06B460122D4
:10B5700003210F20FFF794FF684600780821084058
:10B5800000280BD0FFF74EFEFF2501352A4600218B
:10B590000D2000F0D3F80020C04338BD0020FCE7A8
:10B5A00010B50446224601210A2000F0D8F810BD4B
:10B5B00070B5054600211A20FFF752FF0446240DFE
:10B5C00024052803000B0443224600211A2000F022
:10B5D000C6F870BD10B50446224602492E2000F080
:10B5E000ADF810BD0418000038B504466B460122C2
:10B5F00003210420FFF754FF002C16DD2246002112
:10B600000C2000F09BF86946087810210843009050
:10B610000F488069090608430D4988616B4601227D
:10B620000321042000F0B0F810E0694608781021EA
:10B630008843009006488069090688430449886168
:10B640006B4601220321042000F09EF838BD000063
:10B650008801002010B5044622460021182000F081
:10B660006DF810BDF8B504460025002000900026B6
:10B670000220204000280AD0802000906B46012242
:10B6800000210D2000F080F801211D480173E00722
:10B69000C00F002826D0694608780621084300908C
:10B6A0006B46012200210D2000F06EF803210F20CF
:10B6B000FFF7BEFE06468120C0003040002801D1C1
:10B6C00000251AE0402000906B46012200210D2049
:10B6D00000F05AF80020FFF78DFD002108480173A3
:10B6E0004D1E0AE0694608780221084300906B4627
:10B6F000012200210D2000F047F82846F8BD000087
:10B70000A80100201CB501AB012203210F20FFF787
:10B71000C7FE6946087980210840694609794022B8
:10B7200011404900884208D0012000906B46012258
:10B7300003210D2000F028F800BF1CBDF8B5054618
:10B740000E4614466846047021124170B1B2A8B288
:10B750006B46022200F018F807463846F8BDFEB5E1
:10B7600006460F461446002503E069464C55240A58
:10B770006D1C042DF9DBB9B2B0B26B46042200F0A7
:10B7800003F801900198FEBDFFB581B006460C4656
:10B7900017460025002C07D180203043C2B229462D
:10B7A0006D1C6846425419E0C0203043C2B228469E
:10B7B0006D1C69460A547F2C03DC28466D1C0C5412
:10B7C0000CE0E0B28021084329466D1C6A465054C3
:10B7D0006004020E28466D1C69460A54A8B23A4617
:10B7E0006946049B00F0EAF905B0F0BD70B5044667
:10B7F0000E461546281901218902884202DD0020E3
:10B80000C04370BDA21E334629460920FFF7BCFF86
:10B810000020F6E770B504460D460648006920434F
:10B82000A90508430646324600210820FFF797FF86
:10B83000002070BD8801002038B504466B46012207
:10B840000E212B20FFF72CFE6846007841094901A4
:10B850000091E106C90E68460078014300916B46ED
:10B8600001220E212B20FFF78FFF38BD70B5014656
:10B87000002006E00A541E06140A34431B0A22461E
:10B88000401C0428F6DB70BD13B50C4601231A4694
:10B8900069460248FCF748FE00981CBDDC160020F3
:10B8A0007CB500210C460D466846FFF734FE0426A1
:10B8B00008E0220E28021043240205466846805DF7
:10B8C0000443761E002EF4DA204629467CBD7CB562
:10B8D00000210C460D466846FFF72CFE042608E0C2
:10B8E000220E28021043240205466846805D044368
:10B8F000761E002EF4DA204629467CBDFBF700FBBD
:10B90000FEF746FAFDF712FAFDF7F0FAFDF7F4F943
:10B91000FDF732FBFDF706FBFDF7A6F9FEF788F809
:10B92000FDF76AF8FAF75AF9FAF71CF90721FF2030
:10B930004130FFF745FC334800880A21484332492B
:10B9400008800122110305200007FBF7C4FAC82272
:10B950002E492F48FCF772FD002801D0FAF780F934
:10B960004FE02C480078002849D0FEF711FA00205B
:10B9700028490870284801880088401C264A108001
:10B980007D20C000814222DAFAF7E2FB23490870E9
:10B99000084600780F280DDD012211032048FBF72F
:10B9A0009AFAFEF787FA0022012109031C48FBF7E7
:10B9B00092FA0CE0012251031948FBF78CFAFEF7CA
:10B9C00079FA0022012149031548FBF784FAFCF7B4
:10B9D0003FFF0D480088002804DD0B480088401E0A
:10B9E000094908800F48007800280AD106480088D5
:10B9F000002806D101210846FBF7EEFC01E0FCF728
:10BA000027FFAEE75801002068010020EC0C002061
:10BA1000DC160020490100207201002048010020AE
:10BA2000000400504500002000B585B01748FBF722
:10BA30000CFB14216846F9F7CEFB15480090032053
:10BA4000019000200290694605200007FBF744F9A9
:10BA500069461048FBF740F969460F48FBF73CF987
:10BA600001210846FBF7B8FCFF200130FBF786FCFC
:10BA70000A48006804210843084908608815FBF754
:10BA80008FFCFBF795FC05B000BD000054160020AC
:10BA9000FFFF00000004005000080050007000404C
:10BAA00010B5012292021B491B48FAF710F91948F8
:10BAB00000881A4988422CD008461649088004207C
:10BAC0008880FF20F530C8800A2008810020488146
:10BAD0001E20C04388810120C8810020088408827C
:10BAE00048828882C882088388834320C8860220CF
:10BAF00008877820488701208887C8870021054863
:10BB0000403001844184818400200249C88300F0D0
:10BB10003BF810BDB40D002000FC0008AA55000041
:10BB200070B504460D460021102005263607B06288
:10BB300000BF0DE0685C134EF06000BF11488068E4
:10BB4000C007C00F0028F9D00E48C0681870491C03
:10BB5000A142EFDB00210DE000200A4EF06000BFA3
:10BB600008488068C007C00F0028F9D00548C068A1
:10BB70005854491C9142EFD3102005263607B06176
:10BB8000002070BD0030014010B5002472B60121C4
:10BB900089020848FAF780F80446002C06D00122F2
:10BBA000920205490348FAF769F9044662B620464D
:10BBB00010BD000000FC0008B40D002070B5044664
:10BBC0000D460021102005263607B06200BF0CE0AC
:10BBD000685C124EF06000BF10488068C007C00F5C
:10BBE0000028F9D00D48C068491CA142F0DB0021B3
:10BBF0000CE0585C094EF06000BF08488068C00740
:10BC0000C00F0028F9D00548C068491C9142F0D304
:10BC1000102005263607B061002070BD00300140BD
:10BC20000000010203040005405C0000A05C040069
:10BC3000C06C0800805C0400E03F1E00E07D1E0038
:10BC400007A9022570889B880A00160001000600DB
:10BC50000100020087008D002D001A3152001A33B6
:10BC60009A001A351D011A376B003B31BE003B3379
:10BC70005E013B3596023B37000099599959EB51CB
:10BC80008F421E45142E0080EB51F5283333E13AE4
:10BC9000703DE13AC235852BC2353333C235C235EA
:10BCA000AE47E13A5138A33051380000000000009F
:10BCB0000000010203040607080900000000010259
:10BCC0000304030406080C1018203000ECBC000824
:10BCD0000000002088010000D459000828BD000899
:10BCE00088010020801A0000C6AA0008211307045A
:10BCF000380D091E080540082609104008560A1389
:10BD00001D043B08BE0596D8BC401008042FC8424D
:10BD1000011501020214130909120202C5817B8C6C
:08BD20000ADA0147522000007D
:04000005080050C1DE
:00000001FF
